:020000020000FC
:020000040000FA
:1000000008000500080805000800050008080500AC
:10001000080D04000200020F020D020D020F020E75
:100020000200020E020F020F020F020E020E020E5B
:10003000020F02010201020E020102040200020488
:10004000020F02000201020F02010201020F020F61
:10005000020E090D08080400020C020A0209020D32
:10006000020A0209020C0209020C0209020C020A2D
:1000700002090209020A020A020A0208020A02002E
:10008000020E0209020E02090200020E0209020E0D
:1000900002090200020A020A020A0209020C020A0A
:1000A0000200020002000200020002000908080823
:1000B00004000208020002080209020E0209020EF0
:1000C0000209020E0208020E0208020F020E0204CA
:1000D00002020209020E020D020A020902080208C7
:1000E00002000209020802000204020002080909D3
:1000F0000000000000000000000000000000000000
:00000001FF
